:1074000080E189BD82E189BD09B400FEFDCF089508
:10741000D0D569F08091E9008F931092E900A5D44E
:1074200083FF01C024D58F9187708093E900089570
:107430008EEF0090E10008220092E1000895F20131
:10744000F999FECFF2BDE1BD0895F9DFF89A80B554
:1074500008C0F5DF1FBA80BD0FB6F894FA9AF99A02
:107460000FBE31962F010895E0E0F0E085919491F0
:107470000196089580EE8BB98BEA34D01092890082
:107480008AEF8093880082E080936F0083E080938E
:107490008100E7E5F7E785913AD0E336E1F781E04F
:1074A0008093D7008AE482BF1092D8001092E20045
:1074B0001092DA001092E10080E808D019BC1EBAE0
:1074C0001092E00068D489E059D481E98093D80013
:1074D0000895A3E6B1E090E81AD08D939A95E1F76C
:1074E000089586E008D010C083E005D08F2F0FD01C
:1074F0008E2F0DD080E05F9A5A9809C005D085E0A4
:10750000FADF05D080FDFDCF5A9A5F9808958EBDB1
:107510008DB587FFFDCF8EB508958FE08221E9F705
:10752000F3DFE3E6F6E090EB5C98892FF0DF80E193
:10753000EEDF5C9A8191EBDF83E68E278F77D1F7C0
:107540009395983B89F70895E3E6F1E094FC36C003
:1075500096FC4DC090FE089596849920D1F3F8943E
:10756000C089D78520E030E080E090E4AFEFBFEF46
:10757000119689199040E0F72D01BD4F8D0127FD2F
:1075800013C0E0E0F8E011928EE7819392E4E117F6
:1075900091939AE508F092E4E334C9F7819310825D
:1075A000BFDFFE012196A0DF94DFF90105D5205849
:1075B0003F4F040D151D9A9411F714C28301282D15
:1075C00060906C0170906B0143D019F48823C1F76F
:1075D0000895380188243CD0C9F580916A0182174A
:1075E00009F4830160906E0170906D01F4CF80E426
:1075F000982E60906E0170906D012AD059F4882306
:10760000B1F708959FEF95FC03C092FE089591E0B5
:1076100097FB890E662477248301222719D0B1F4C1
:107620008823A1F380916A0136F0881650F48217FE
:1076300030F0213003C0881520F4281710F483019E
:10764000282F60906E0170906D01E8CF3801822E76
:10765000F3014ADF3EDFC3E6D1E0E0E5F7E709905A
:107660008591081621F4E735D1F7088080104CCFBA
:10767000C9E031DFCA95E9F7D0E194FC55C096FC2A
:1076800037C092FE1AC0C3E6D2E0E3E6F6E098E027
:1076900088E78E0F00840192E817E1F7884F099080
:1076A0000192E817E1F7C858DF4F9A9589F735DF5F
:1076B000C85FD340C33E49F749C0C3E6D6E0EBE517
:1076C000FAE098E08E2F885702900086E817E1F7DD
:1076D00038960A900292E817E1F73897C857D040D9
:1076E0009A9581F71ADFC850DC4FC33E41F72EC090
:1076F000A3EEB6E0E3E6F6E09AE0C6E00D90808106
:107700008025807F802582958193A336B90709F46F
:10771000B2E0E336F90709F4F2E0E336FC0771F76B
:10772000FCDEDA9529F712C0A3EEB9E0E3E6FAE051
:1077300092E00E90829180258F70802582958083C3
:10774000E336F907B1F7E9DEDA9571F7882708958E
:1077500041524455424F59D5F08D14A1C881CFD91B
:10776000F1AF000000FFFFCFCFFFFFFFFFCFCFFF44
:10777000FF0000FE067E7E06FE46565616FE0656A4
:10778000461EFE3F61E9E3FFE3EBE3FFE3EBE3FFCC
:04779000E16B3F006A
:10779400120110010200000841233600010000001C
:1077A400000109023E0002010080320904000001C8
:1077B4000202010005240010010424020405240629
:1077C4000001070582030800FF09040100020A0002
:1077D40000000705040210000107058302100001E0
:1078000011241FBE04B714BE88E18093600010925B
:1078100060008EEF9AE09EBF8DBF222433242101A9
:107820003101410180E88AC00F928F939F931F928C
:107830000FB60F9211244F936F938091DA0080FF5F
:1078400037C023C00F920FB68F939F93EF93FF9390
:1078500088278093850080938400E0E5F1E09281A1
:10786000907261F490818917980B908309F45D9A66
:1078700091818917980B918309F4289A239411F424
:107880008315381EFF91EF9154C08091D80080FF7E
:107890000FC08091DA008E7F8093DA008091D9004A
:1078A00080FF04C0ADDD81E08EBB02C019BC1EBAF2
:1078B0008091E10080FF0BC05BD280FF08C05BD2EB
:1078C0008091D800806202DE19BC85E08EBB809179
:1078D000E10084FF1AC04CD284FF17C091DD809173
:1078E000D8008F7DF3DD8FEEA4DD42D28F7E8160E4
:1078F00045D280915301882331F48091E30087FDC4
:1079000002C081E001C084E08EBB8091E10083FF72
:107910000CC02ED283FF09C087EF8BDD82E08EBBC7
:107920001092530185DD27D236D26F914F910F907F
:107930001F909F918F910FBE0F90189580936100BB
:1079400010926100B1E0B5BF82E085BF87E084B9E5
:1079500081E785B917B8469A10BA80EC81BB84EAF2
:107960008BB984EF8AB980E58CBDBDBDA0E0E4E9A8
:10797000F7E705900D92A035E1F71D92BB30E9F7CE
:1079800001FD06C0000004C01E9B02C06DDD51F564
:1079900071DD78945DDE71F0ABE9B7E0E3E6F7E71F
:1079A00090E105900D929A95E1F7A059BF4FE33908
:1079B000B9F7B7DD54D02CDD80915201807871F495
:1079C00083B180958077369B84607F997E9B8160B0
:1079D000982E18DE8110B8DD90FC02C0332052F7DB
:1079E00043DD41F3F89489EB7DDD81E08093E00095
:1079F00010926F0010928100109285001092840006
:107A000081E085BF15BE289A289A289A5D9A289AFF
:107A10000C940000A8D107C05BD102C0CAD239F0D3
:107A2000A4D182FFFBCF85FFF7CF8091F1000895AD
:107A3000082E83E099D185FD07C08ED102C0B9D24E
:107A400069F093D180FFFBCF0092F1008091520149
:107A5000807221F45D9884E680935001089583D16B
:107A600082FF38C180915201807221F4289884E607
:107A700080935101CFDF182F853431F422248EE713
:107A8000382EDDDC8DE00FC1843511F4C3DFFACF71
:107A90008C34C1F38035B1F3843721F484E4C8DF3A
:107AA00080E001C1813611F489E5FDC0813429F4FB
:107AB000B1DF582EAFDF482EE5CF803711F483E5D4
:107AC000F2C0833539F4E0E5F7E78591B1DFE735BA
:107AD000E1F7EAC0863521F481E3AADF89E3E3C058
:107AE000863781F481E37F9B8E5F7E9B8F5FA0DF73
:107AF00081E41C9B885F369B8C5F1D9B8E5F1E9B69
:107B00008F5FD1C08837A9F485DF80935201289A0E
:107B100084FD28985D9A83FD5D98289A81FD2898B8
:107B2000289A82FD2898289A80FD289887FD882425
:107B3000A9CF8A3649F48FE9DEDCC3E0E8DC78DFE0
:107B4000CA95E1F7E1DCB0C0833731F487E870DF34
:107B500085E96EDF8EE1A7C0853639F4E0E8F3E70A
:107B60003ED2E058F040E0F78DCF823631F489E51F
:107B70005FDF80E05DDF80E896C0823419F08736F1
:107B800009F07DC0332446DFD82F44DFC82F42DF01
:107B9000082F8354843008F085C0063411F4440C57
:107BA000551CF20110926F001736B9F4033489F4B2
:107BB00083E09BDCACDC8EB51EBC3ADF0DB42197B4
:107BC000D1F7A2DC08C0063411F4859101C03DDC78
:107BD0002FDF2197C2F72F014AC00334A9F4E11126
:107BE00004C07FDC88ED81DC89DC7BDC82E07DDC2D
:107BF00011DF0DB48EBDCA95D9F7319689DC7EDCD4
:107C0000DA9569F72F0131C00634F1F49F01F4379A
:107C1000D8F4E5D119C0FEDE063461F4C0FB46F0AD
:107C2000F43728F4182E81E087BFE89511243296A6
:107C3000082E0AC0043439F4DF01B370AD59B94FCE
:107C40008D93319601C005DC21972AF7043431F475
:107C50002F01F370FE2B49F464DC07C0063429F4CD
:107C60002F01F901F43708F4B8D18DE0E1DE0634D4
:107C700011F45694479482E080936F0015C08237C8
:107C8000E1E049F08634E0E031F08E34E3E019F0D1
:107C9000813531F4E2E0F0E089E087BF849103C0F0
:107CA0008B3111F08FE3C4DE83E0BFDB55D095FF4D
:107CB00003C009C07ED171F058D080FFFBCF4CD0FB
:107CC00002C077D139F051D080FFFBCF84E0ADDB2B
:107CD0008BE743C00895E4E5F1E067E090915B0134
:107CE00080915C01913231F0913AE1F58132D1F528
:107CF0005ED181C0823271F48191805B8191844038
:107D000089F580915D0180FD2DC0F89481E080931C
:107D1000E00076CD803231F54AD14BD1E9F08530A3
:107D2000D9F023D083FD18C082FFF7CF04C07DDED9
:107D30008193615031F09091F3008091F200892B92
:107D4000B1F7C6DF611549F704C033D129F085309A
:107D500019F00BD080FFF9CF8EE79091E8008923CE
:107D60008093E800089584E060DB8091E800089546
:107D70008091E2000895FCDF8E7F80618093E200B5
:107D8000089582E061EC09D083E061E802D084E0EC
:107D900060E842E103C080E060E042E046DB81E071
:107DA00007D01092ED006093EC004093ED00089531
:107DB0009091EB00892B8093EB00089560E0923066
:107DC00029F0913029F4E0E062E102C0E2E16EE3E3
:107DD000F1E0089580915B0188234CF402C0E9D062
:107DE000C1F3C3DF82FFFBCF73CFE3D091F3BDDFDD
:107DF00080FFFBCFB1CF40916101509162014617E6
:107E0000510520F0462F611509F4A6DF50E022C08D
:107E1000D0D061F1853051F1A8DF83FD59CFA5DFC6
:107E200082FD21C080FF16C03091F3002091F20046
:107E300006C081918093F10041502F5F3F4F411563
:107E400019F028303105A8F350E02830310509F445
:107E500051E082DF4115E1F65523D1F604C0A9D0E7
:107E600029F0853019F081DF82FFF9CF31CFEBE5C2
:107E7000F1E0DBDD8193E336E1F72DDF76DF83FF91
:107E800091C080915B0190915C01913009F170F09B
:107E90009330F1F0953009F444C0963009F456C09F
:107EA000983009F460C0993059F767C0823841F7BB
:107EB00080915F01B9DA2091EB001092E90077D050
:107EC0002295269521702093F1001092F10052C066
:107ED000882311F08230A1F68F71823089F680916B
:107EE0005D018823D1F420915F01277049F220932E
:107EF000E9008091EB0080FF10C0933011F480E224
:107F00000BC080E155DF81E0880F2A95E9F7809367
:107F1000EA001092EA0088E04BDF1092E90047D0B7
:107F20002AC0882391F410915D0110680FB7F8946E
:107F30003ED050DF1ADF80FFFDCF1093E3001038F2
:107F400083E009F482E08EBB0FBF2CC080588230E2
:107F500048F580915D0190915E0130DF603011F154
:107F600026D049DF1FC08038E9F421D08091530129
:107F70008093F100F1DE2EDF15C0882399F49091F3
:107F80005D01923078F49093530111D023DF8091FA
:107F90005301882321F48091E30091E087FD94E070
:107FA0009EBBEFDEE2DE83FF089580E201DF87EF14
:107FB000D4CE8EB388230895A3E6B1E0F437B8F4A5
:107FC0000ED090E40D901D9081E087BFE895329629
:107FD0009A95C1F71124E058F04085E001C083E094
:107FE00001D081E187BFE89507B600FCFDCF089579
:067FFA003139DFCFFBDC92
:040000030000740085
:00000001FF
